:100000000C9481000C94A4000C94A4000C94A40003
:100010000C94A4000C94A4000C94A4000C94A400D0
:100020000C94A4000C94A4000C94A4000C94A400C0
:100030000C94A4000C94A4000C94A4000C94A400B0
:100040000C94A4000C94A4000C94A4000C94A400A0
:100050000C94A4000C94A4000C94A4000C94A40090
:100060000C94A4000C94A4000C94A4000C94A40080
:100070000C94A4000C94A4000C94A4000C94A40070
:100080000C94A4000C94A4000C94A4000C94A40060
:100090000C94A4000C94A4000C94A4000C94A40050
:1000A0000C94A4000C94A4000C94A4000C94A40040
:1000B0000C94A4000C94A4000C94A4000C94A40030
:1000C0000C94A4000C94A4000C94A4000C94A40020
:1000D0000C94A4000C94A4000C94A4000C94A40010
:1000E0000C94A40005A84CCDB2D44EB93836A90260
:1000F0000C50B9918688083CA6AAAA2ABE00000026
:10010000803F11241FBECFEFD1E2DEBFCDBF00E0A4
:100110000CBF84B78093000314BE0FB6F894A89563
:1001200080916000886180936000109260000FBE33
:1001300023E0A0E0B2E001C01D92A030B207E1F7D9
:100140000E9409010C9450040C9400008093080153
:100150000895A8E0B1E08C938FEF80BBEBE0F1E075
:1001600080818D7F808361BB80818F7E808385E0ED
:100170008A95F1F700008081806180831C928081E4
:100180008260808311BA0895A8E0B1E08C9310BA20
:1001900011BAEBE0F1E080818B7F808380818F7EDC
:1001A000808385E08A95F1F700008FB1908190619E
:1001B00090831C929081946090839FEF90BB11BAC2
:1001C00095E09A95F1F7000008950F931F93CF9350
:1001D00000E012E0C0E0F80161918F018C2F817086
:1001E0000E94A900CF5FCF3FB1F760E080E00E949E
:1001F000A90060E081E00E94A9008FE39CE90197DB
:10020000F1F700C0000090E080E0CF911F910F91C6
:10021000089500D000D0CDB7DEB7F8948FEF80BB43
:100220008093070180930A0111BA1092080110927D
:100230000B0180910B01826080930B0180910B0177
:10024000846080930B0180910B01806180930B018E
:1002500080910B01816080930B018FE891E0019701
:10026000F1F700C0000080910B018E7F80930B019D
:1002700000E012E01E821D82AD81BE81CD01B0E0A2
:10028000A0E089839A83AB83BC83BC01CD010E942B
:10029000C50220E030E04FE753E469837A838B8323
:1002A0009C8369817A818B819C810E941D0228ED4B
:1002B0003FE049EC50E469837A838B839C836981B6
:1002C0007A818B819C810E94530369837A838B831B
:1002D0009C8369817A818B819C810E94C00320E08C
:1002E00030E04FEF52E469837A838B839C8369818A
:1002F0007A818B819C810E94530320E030E04FEF94
:1003000052E469837A838B839C8369817A818B81B0
:100310009C810E94B10169837A838B839C8369816C
:100320007A818B819C810E948F02F80161938F01F9
:100330008D819E8101969E838D838115914009F068
:100340009BCF789488E19EE00FB6F894A8958093AF
:1003500060000FBE90936000A8950E94E500FCCF5E
:100360005058BB27AA270E94C8010C9419030E9469
:100370000B0338F00E94120320F039F49F3F19F468
:1003800026F40C9408030EF4E095E7FB0C940203AA
:10039000E92F0E942A0358F3BA17620773078407EC
:1003A000950720F079F4A6F50C944C030EF4E09533
:1003B0000B2EBA2FA02D0B01B90190010C01CA011F
:1003C000A0011124FF27591B99F0593F50F4503ECA
:1003D00068F11A16F040A22F232F342F4427585FBC
:1003E000F3CF469537952795A795F0405395C9F7D4
:1003F0007EF41F16BA0B620B730B840BBAF091508C
:10040000A1F0FF0FBB1F661F771F881FC2F70EC02A
:10041000BA0F621F731F841F48F4879577956795FD
:10042000B795F7959E3F08F0B0CF9395880F08F0E9
:100430009927EE0F9795879508950E9431020C94A5
:1004400019030E94120358F00E940B0340F029F494
:100450005F3F29F00C94020351110C944D030C944E
:1004600008030E942A0368F39923B1F3552391F3FB
:10047000951B550BBB27AA2762177307840738F013
:100480009F5F5F4F220F331F441FAA1FA9F335D070
:100490000E2E3AF0E0E832D091505040E695001C24
:1004A000CAF72BD0FE2F29D0660F771F881FBB1FDE
:1004B000261737074807AB07B0E809F0BB0B802DBC
:1004C000BF01FF2793585F4F3AF09E3F510578F0E8
:1004D0000C9402030C944D035F3FE4F3983ED4F375
:1004E000869577956795B795F7959F5FC9F7880FBC
:1004F000911D9695879597F90895E1E0660F771F0E
:10050000881FBB1F621773078407BA0720F0621B9E
:10051000730B840BBA0BEE1F88F7E09508950E94C9
:1005200096026894B1110C944D0308950E94320311
:1005300088F09F5798F0B92F9927B751B0F0E1F0A4
:10054000660F771F881F991F1AF0BA95C9F714C054
:10055000B13091F00E944C03B1E008950C944C032B
:10056000672F782F8827B85F39F0B93FCCF386958D
:1005700077956795B395D9F73EF4909580957095EA
:1005800061957F4F8F4F9F4F0895E89409C097FB67
:100590003EF490958095709561957F4F8F4F9F4F5A
:1005A0009923A9F0F92F96E9BB279395F69587959E
:1005B00077956795B795F111F8CFFAF4BB0F11F461
:1005C00060FF1BC06F5F7F4F8F4F9F4F16C0882308
:1005D00011F096E911C0772321F09EE8872F762F3E
:1005E00005C0662371F096E8862F70E060E02AF07F
:1005F0009A95660F771F881FDAF7880F969587956B
:1006000097F9089597F99F6780E870E060E0089592
:100610009FEF80EC089500240A941616170618061A
:100620000906089500240A941216130614060506F6
:100630000895092E0394000C11F4882352F0BB0F87
:1006400040F4BF2B11F460FF04C06F5F7F4F8F4FEA
:100650009F4F089557FD9058440F551F59F05F3F25
:1006600071F04795880F97FB991F61F09F3F79F0D4
:1006700087950895121613061406551FF2CF469556
:10068000F1DF08C0161617061806991FF1CF8695D8
:100690007105610508940895E894BB2766277727BC
:1006A000CB0197F908950E9466030C9419030E94E8
:1006B0000B0338F00E94120320F0952311F00C94E4
:1006C00002030C94080311240C944D030E942A0386
:1006D00070F3959FC1F3950F50E0551F629FF00195
:1006E000729FBB27F00DB11D639FAA27F00DB11DAE
:1006F000AA1F649F6627B00DA11D661F829F222737
:10070000B00DA11D621F739FB00DA11D621F839FBD
:10071000A00D611D221F749F3327A00D611D231F93
:10072000849F600D211D822F762F6A2F11249F57E1
:1007300050409AF0F1F088234AF0EE0FFF1FBB1FE4
:10074000661F771F881F91505040A9F79E3F5105A3
:1007500080F00C9402030C944D035F3FE4F3983E49
:10076000D4F3869577956795B795F795E7959F5F4D
:10077000C1F7FE2B880F911D9695879597F90895DF
:100780009F930E94CA030F9007FCEE5F0C94F30343
:100790000C9408030E943203D8F3E894E0E0BB27EE
:1007A0009F57F0F02AED3FE049EC06C0EE0FBB0F7B
:1007B000661F771F881F28F0B23A62077307840705
:1007C00028F0B25A620B730B840BE3959A9572F77B
:1007D000803830F49A95BB0F661F771F881FD2F7B9
:1007E00090480C940904EF93E0FF07C0A2EA2AEDB9
:1007F0003FE049EC5FEB0E94C8010E9419030F9093
:10080000039401FC9058E4EEF0E00C9415049F3F33
:1008100031F0915020F4879577956795B795880FBB
:10082000911D9695879597F908959F938F937F9340
:100830006F93FF93EF939B01AC010E945303EF91E1
:10084000FF910E9429042F913F914F915F910C9449
:100850005303DF93CF931F930F93FF92EF92DF9297
:100860007B018C01689406C0DA2EEF010E946603BA
:10087000FE01E894A5912591359145915591A6F3F6
:10088000EF010E94C801FE019701A801DA9469F7FF
:10089000DF90EF90FF900F911F91CF91DF9108951E
:0408A000F894FFCFFA
:00000001FF
